:020000040000fa
:080000000002040000000000f2
:020000040000fa
:100400006f86200020bf200000018800000000004f
:10041000050007000c000700f202020000000000c7
:100420000040da000000fe004440a9000000200067
:100430000000e0000300320000002000a00188005e
:100440004440a80000000600803220000100200087
:100450001600370062004000e080480091018800eb
:100460009001ba0062004000e080480091018800dd
:100470009002ba0062004000e08048000002eb00f9
:100480006028e10005003a008301e900070033001d
:10049000038009000059eb00040037006128e100e7
:1004a000010032000082eb00050007009101880086
:1004b0001001ba000200e000e6ff3a00000005006b
:1004c000910188008002780062004000e0804800ce
:1004d0003559ba008301e900080032002559ba00f5
:1004e0008301e900050032000400e000f4ff32005f
:1004f00015d9ba008301e900f1ff3a0000000600b7
:10050000881f78008a1f78004400f800080f200038
:10051000280288000004900010059000a0009000c0
:1005200030019000c00190000300ca000280ca00a0
:100530000030cb001a00cd004604c3000100ca0001
:100540004604c0001e04c0000605c0000100cd0026
:1005500021009800050d7800eaba9700052578007b
:100560004400f9004f0578004f04780000000600b1
:10057000801f78004000b0000008eb004f007800ba
:10058000801f7800100090000018eb000018eb00ae
:100590000008eb004f007800000006004400f8005f
:1005a000020f200022028800910078003000ca006b
:1005b0003080ca000000cb002080ca000000cb00c1
:1005c0003100cd004000ca000000cb000000cb008d
:1005d0000010cb003100cd001180cc004400f900a8
:1005e000000006000000fa0000852000b0428800ec
:1005f000a0bf2000c042880060852000dcff07000b
:1006000090992500004388009099210010438800ac
:10061000608f200020438800618520000086200034
:10062000deff070080eb2500f0428800b09f23002a
:10063000e04288000000eb00401688006085200042
:10064000afff0700d042800050168800f9ff370046
:020000040000fa
:1000080046030000460300004603000046030000c4
:1000180046030000460300004603000046030000b4
:1000280046030000460300004603000046030000a4
:100038004603000046030000460300004603000094
:020000040000fa
:020000040000fa
:10065000600800000600000002000000000000002a
:1006600000000000560800000a0000000000000022
:10067000500800000600000000000000fa0b000017
:0c06800006000000000000000000000068
:020000040000fa
:04068c000000fe006c
:00000001FF
